 popframe004

 Timestamp is 5d5a510d (reproducible build file hash)

 Preferred load address is 0000000180000000

 Start         Length     Name                   Class
 0001:00000000 000036d0H .text$mn                CODE
 0001:000036d0 00000036H .text$mn$00             CODE
 0001:00003706 00000092H .text$x                 CODE
 0002:00000000 000001b8H .idata$5                DATA
 0002:000001b8 00000038H .00cfg                  DATA
 0002:000001f0 00000008H .CRT$XCA                DATA
 0002:000001f8 00000008H .CRT$XCZ                DATA
 0002:00000200 00000008H .CRT$XIA                DATA
 0002:00000208 00000008H .CRT$XIC                DATA
 0002:00000210 00000008H .CRT$XIZ                DATA
 0002:00000218 00000008H .CRT$XLA                DATA
 0002:00000220 00000008H .CRT$XLZ                DATA
 0002:00000228 00000008H .CRT$XPA                DATA
 0002:00000230 00000008H .CRT$XPZ                DATA
 0002:00000238 00000008H .CRT$XTA                DATA
 0002:00000240 00000010H .CRT$XTZ                DATA
 0002:00000248 00000000H .gehcont$y              DATA
 0002:00000248 00000000H .gfids$y                DATA
 0002:00000250 000021b0H .rdata                  DATA
 0002:00002400 00000000H .rdata$CastGuardVftablesA DATA
 0002:00002400 00000000H .rdata$CastGuardVftablesC DATA
 0002:00002400 00000028H .rdata$T                DATA
 0002:00002428 000000a4H .rdata$voltmd           DATA
 0002:000024cc 0000031cH .rdata$zzzdbg           DATA
 0002:000027e8 00000008H .rtc$IAA                DATA
 0002:000027f0 00000008H .rtc$IZZ                DATA
 0002:000027f8 00000008H .rtc$TAA                DATA
 0002:00002800 00000008H .rtc$TZZ                DATA
 0002:00002808 00000004H .tls                    DATA
 0002:0000280c 00000004H .tls$                   DATA
 0002:00002810 00000008H .tls$ZZZ                DATA
 0002:00002818 00000338H .xdata                  DATA
 0002:00002b50 00000410H .edata                  DATA
 0002:00002f60 00000064H .idata$2                DATA
 0002:00002fc4 00000014H .idata$3                DATA
 0002:00002fd8 000001b8H .idata$4                DATA
 0002:00003190 00000476H .idata$6                DATA
 0003:00000000 00000080H .data                   DATA
 0003:00000080 0001b3a8H .bss                    DATA
 0004:00000000 00000420H .pdata                  DATA

  Address         Publics by Value              Rva+Base               Lib:Object

 0000:00000000       __AbsoluteZero             0000000000000000     <absolute>
 0000:00000000       ___safe_se_handler_count   0000000000000000     <absolute>
 0000:00000000       ___safe_se_handler_table   0000000000000000     <absolute>
 0000:00000000       __arm64x_extra_rfe_table   0000000000000000     <absolute>
 0000:00000000       __arm64x_extra_rfe_table_size 0000000000000000     <absolute>
 0000:00000000       __arm64x_native_entrypoint 0000000000000000     <absolute>
 0000:00000000       __arm64x_redirection_metadata 0000000000000000     <absolute>
 0000:00000000       __arm64x_redirection_metadata_count 0000000000000000     <absolute>
 0000:00000000       __dynamic_value_reloc_table 0000000000000000     <absolute>
 0000:00000000       __enclave_config           0000000000000000     <absolute>
 0000:00000000       __guard_check_icall_a64n_fptr 0000000000000000     <absolute>
 0000:00000000       __guard_eh_cont_count      0000000000000000     <absolute>
 0000:00000000       __guard_eh_cont_table      0000000000000000     <absolute>
 0000:00000000       __guard_fids_count         0000000000000000     <absolute>
 0000:00000000       __guard_fids_table         0000000000000000     <absolute>
 0000:00000000       __guard_iat_count          0000000000000000     <absolute>
 0000:00000000       __guard_iat_table          0000000000000000     <absolute>
 0000:00000000       __guard_longjmp_count      0000000000000000     <absolute>
 0000:00000000       __guard_longjmp_table      0000000000000000     <absolute>
 0000:00000000       __hybrid_auxiliary_iat     0000000000000000     <absolute>
 0000:00000000       __hybrid_auxiliary_iat_copy 0000000000000000     <absolute>
 0000:00000000       __hybrid_code_map          0000000000000000     <absolute>
 0000:00000000       __hybrid_code_map_count    0000000000000000     <absolute>
 0000:00000000       __x64_code_ranges_to_entry_points 0000000000000000     <absolute>
 0000:00000000       __x64_code_ranges_to_entry_points_count 0000000000000000     <absolute>
 0000:00000100       __guard_flags              0000000000000100     <absolute>
 0000:00000000       __ImageBase                0000000180000000     <linker-defined>
 0001:00000000       ?CallVoidMethod@JNIEnv_@@QEAAXPEAV_jobject@@PEAU_jmethodID@@ZZ 0000000180001000 f i libpopframe004.obj
 0001:00000024       ?NewObject@JNIEnv_@@QEAAPEAV_jobject@@PEAV_jclass@@PEAU_jmethodID@@ZZ 0000000180001024 f i libpopframe004.obj
 0001:0000004c       ?SetEventNotificationMode@_jvmtiEnv@@QEAA?AW4jvmtiError@@W4jvmtiEventMode@@W4jvmtiEvent@@PEAV_jobject@@ZZ 000000018000104c f i libpopframe004.obj
 0001:00000058       ?TranslateError@@YAPEBDW4jvmtiError@@@Z 0000000180001058 f   libpopframe004.obj
 0001:00000378       ?nsk_jni_check_exception@@YAHPEAUJNIEnv_@@QEBDH@Z 0000000180001378 f   libpopframe004.obj
 0001:000004bc       ?nsk_jni_lverify@@YAHHPEAUJNIEnv_@@HQEBDH1ZZ 00000001800014bc f   libpopframe004.obj
 0001:000009a8       Agent_Initialize           00000001800019a8 f   libpopframe004.obj
 0001:00000b68       Agent_OnAttach             0000000180001b68 f   libpopframe004.obj
 0001:00000b68       Agent_OnLoad               0000000180001b68 f   libpopframe004.obj
 0001:00000b70       FramePop                   0000000180001b70 f   libpopframe004.obj
 0001:00000bc4       Java_nsk_jvmti_PopFrame_popframe004_doPopFrame 0000000180001bc4 f   libpopframe004.obj
 0001:00000e4c       Java_nsk_jvmti_PopFrame_popframe004_getResult 0000000180001e4c f   libpopframe004.obj
 0001:00000e54       Java_nsk_jvmti_PopFrame_popframe004_nativeMeth 0000000180001e54 f   libpopframe004.obj
 0001:00000eac       Java_nsk_jvmti_unit_FollowReferences_FollowRefObjects_addRefToVerify 0000000180001eac f   libpopframe004.obj
 0001:00001084       Java_nsk_jvmti_unit_FollowReferences_FollowRefObjects_getTag 0000000180002084 f   libpopframe004.obj
 0001:00001144       Java_nsk_jvmti_unit_FollowReferences_FollowRefObjects_resetRefsToVerify 0000000180002144 f   libpopframe004.obj
 0001:0000114c       Java_nsk_jvmti_unit_FollowReferences_FollowRefObjects_resetTags 000000018000214c f   libpopframe004.obj
 0001:00001190       Java_nsk_jvmti_unit_FollowReferences_FollowRefObjects_setTag 0000000180002190 f   libpopframe004.obj
 0001:000013e8       Java_nsk_share_jvmti_ArgumentHandler_getAgentOptionsString 00000001800023e8 f   libpopframe004.obj
 0001:00001498       Java_nsk_share_jvmti_DebugeeClass_checkStatus 0000000180002498 f   libpopframe004.obj
 0001:00001520       Java_nsk_share_jvmti_DebugeeClass_resetAgentData 0000000180002520 f   libpopframe004.obj
 0001:00001580       Java_nsk_share_jvmti_RedefineAgent_agentStatus 0000000180002580 f   libpopframe004.obj
 0001:0000158c       Java_nsk_share_jvmti_RedefineAgent_isRedefined 000000018000258c f   libpopframe004.obj
 0001:00001598       Java_nsk_share_jvmti_RedefineAgent_redefineAttempted 0000000180002598 f   libpopframe004.obj
 0001:000015a4       MA_checkStatus             00000001800025a4 f   libpopframe004.obj
 0001:00001648       MethodExit                 0000000180002648 f   libpopframe004.obj
 0001:0000169c       __local_stdio_printf_options 000000018000269c f i libpopframe004.obj
 0001:0000187c       exitOnError                000000018000287c f   libpopframe004.obj
 0001:00001930       fprintf                    0000000180002930 f i libpopframe004.obj
 0001:00001974       nativeMeth2                0000000180002974 f   libpopframe004.obj
 0001:00001a18       nsk_jvmti_lverify          0000000180002a18 f   libpopframe004.obj
 0001:00001b08       nsk_jvmti_resetAgentData   0000000180002b08 f   libpopframe004.obj
 0001:00001b88       nsk_jvmti_setFailStatus    0000000180002b88 f   libpopframe004.obj
 0001:00001bc4       nsk_lcomplain              0000000180002bc4 f   libpopframe004.obj
 0001:00001be4       nsk_ldisplay               0000000180002be4 f   libpopframe004.obj
 0001:00001c04       nsk_ltrace                 0000000180002c04 f   libpopframe004.obj
 0001:00001c24       nsk_lvcomplain             0000000180002c24 f   libpopframe004.obj
 0001:00001ddc       nsk_lvdisplay              0000000180002ddc f   libpopframe004.obj
 0001:00001e28       nsk_lverify                0000000180002e28 f   libpopframe004.obj
 0001:00001e84       nsk_lvtrace                0000000180002e84 f   libpopframe004.obj
 0001:00001ee4       nsk_printf                 0000000180002ee4 f   libpopframe004.obj
 0001:00001f0c       nsk_vprintf                0000000180002f0c f   libpopframe004.obj
 0001:00001fc0       printf                     0000000180002fc0 f i libpopframe004.obj
 0001:00002010       resThread                  0000000180003010 f   libpopframe004.obj
 0001:000023f8       suspThread                 00000001800033f8 f   libpopframe004.obj
 0001:00002638       __raise_securityfailure    0000000180003638 f   MSVCRT:gs_report.obj
 0001:0000266c       __report_gsfailure         000000018000366c f   MSVCRT:gs_report.obj
 0001:000028ac       _Init_thread_footer        00000001800038ac f   MSVCRT:thread_safe_statics.obj
 0001:0000290c       _Init_thread_header        000000018000390c f   MSVCRT:thread_safe_statics.obj
 0001:00002974       _Init_thread_notify        0000000180003974 f   MSVCRT:thread_safe_statics.obj
 0001:000029b8       _Init_thread_wait          00000001800039b8 f   MSVCRT:thread_safe_statics.obj
 0001:00002a1c       __GSHandlerCheck           0000000180003a1c f   MSVCRT:gshandler.obj
 0001:00002a3c       __GSHandlerCheckCommon     0000000180003a3c f   MSVCRT:gshandler.obj
 0001:00002ab0       __security_check_cookie    0000000180003ab0 f   MSVCRT:amdsecgs.obj
 0001:00002df0       _DllMainCRTStartup         0000000180003df0 f   MSVCRT:dll_dllmain.obj
 0001:00002e30       __scrt_acquire_startup_lock 0000000180003e30 f   MSVCRT:utility.obj
 0001:00002e6c       __scrt_dllmain_after_initialize_c 0000000180003e6c f   MSVCRT:utility.obj
 0001:00002ea0       __scrt_dllmain_before_initialize_c 0000000180003ea0 f   MSVCRT:utility.obj
 0001:00002eb8       __scrt_dllmain_crt_thread_attach 0000000180003eb8 f   MSVCRT:utility.obj
 0001:00002ee0       __scrt_dllmain_crt_thread_detach 0000000180003ee0 f   MSVCRT:utility.obj
 0001:00002ef8       __scrt_dllmain_exception_filter 0000000180003ef8 f   MSVCRT:utility.obj
 0001:00002f58       __scrt_dllmain_uninitialize_c 0000000180003f58 f   MSVCRT:utility.obj
 0001:00002f88       __scrt_dllmain_uninitialize_critical 0000000180003f88 f   MSVCRT:utility.obj
 0001:00002f9c       __scrt_initialize_crt      0000000180003f9c f   MSVCRT:utility.obj
 0001:00002fe8       __scrt_initialize_onexit_tables 0000000180003fe8 f   MSVCRT:utility.obj
 0001:00003074       __scrt_is_nonwritable_in_current_image 0000000180004074 f   MSVCRT:utility.obj
 0001:0000310c       __scrt_release_startup_lock 000000018000410c f   MSVCRT:utility.obj
 0001:00003130       __scrt_uninitialize_crt    0000000180004130 f   MSVCRT:utility.obj
 0001:0000315c       _onexit                    000000018000415c f   MSVCRT:utility.obj
 0001:00003198       atexit                     0000000180004198 f   MSVCRT:utility.obj
 0001:000031b0       __crt_debugger_hook        00000001800041b0 f   MSVCRT:utility_desktop.obj
 0001:000031b8       __scrt_fastfail            00000001800041b8 f   MSVCRT:utility_desktop.obj
 0001:00003304       _guard_check_icall_nop     0000000180004304 f i MSVCRT:guard_support.obj
 0001:00003308       __security_init_cookie     0000000180004308 f   MSVCRT:gs_support.obj
 0001:000033b4       DllMain                    00000001800043b4 f   MSVCRT:dll_dllmain_stub.obj
 0001:000033d8       ?__scrt_initialize_type_info@@YAXXZ 00000001800043d8 f   MSVCRT:tncleanup.obj
 0001:000033e8       ?__scrt_uninitialize_type_info@@YAXXZ 00000001800043e8 f   MSVCRT:tncleanup.obj
 0001:000033f4       __local_stdio_scanf_options 00000001800043f4 f i MSVCRT:default_local_stdio_options.obj
 0001:000033fc       __scrt_initialize_default_local_stdio_options 00000001800043fc f   MSVCRT:default_local_stdio_options.obj
 0001:00003418       __scrt_get_dyn_tls_init_callback 0000000180004418 f   MSVCRT:dyn_tls_init.obj
 0001:00003420       _RTC_Initialize            0000000180004420 f   MSVCRT:initsect.obj
 0001:0000345c       _RTC_Terminate             000000018000445c f   MSVCRT:initsect.obj
 0001:00003498       __isa_available_init       0000000180004498 f   MSVCRT:cpu_disp.obj
 0001:00003644       _get_startup_argv_mode     0000000180004644 f   MSVCRT:argv_mode.obj
 0001:0000364c       __scrt_is_ucrt_dll_in_use  000000018000464c f   MSVCRT:ucrt_detection.obj
 0001:00003660       memcpy                     0000000180004660 f   vcruntime:VCRUNTIME140.dll
 0001:00003666       memset                     0000000180004666 f   vcruntime:VCRUNTIME140.dll
 0001:0000366c       strchr                     000000018000466c f   vcruntime:VCRUNTIME140.dll
 0001:00003672       __C_specific_handler       0000000180004672 f   vcruntime:VCRUNTIME140.dll
 0001:00003678       __std_type_info_destroy_list 0000000180004678 f   vcruntime:VCRUNTIME140.dll
 0001:0000367e       strlen                     000000018000467e f   ucrt:api-ms-win-crt-string-l1-1-0.dll
 0001:00003684       _initterm                  0000000180004684 f   ucrt:api-ms-win-crt-runtime-l1-1-0.dll
 0001:0000368a       _initterm_e                000000018000468a f   ucrt:api-ms-win-crt-runtime-l1-1-0.dll
 0001:00003690       _seh_filter_dll            0000000180004690 f   ucrt:api-ms-win-crt-runtime-l1-1-0.dll
 0001:00003696       _configure_narrow_argv     0000000180004696 f   ucrt:api-ms-win-crt-runtime-l1-1-0.dll
 0001:0000369c       _initialize_narrow_environment 000000018000469c f   ucrt:api-ms-win-crt-runtime-l1-1-0.dll
 0001:000036a2       _initialize_onexit_table   00000001800046a2 f   ucrt:api-ms-win-crt-runtime-l1-1-0.dll
 0001:000036a8       _register_onexit_function  00000001800046a8 f   ucrt:api-ms-win-crt-runtime-l1-1-0.dll
 0001:000036ae       _execute_onexit_table      00000001800046ae f   ucrt:api-ms-win-crt-runtime-l1-1-0.dll
 0001:000036b4       _crt_atexit                00000001800046b4 f   ucrt:api-ms-win-crt-runtime-l1-1-0.dll
 0001:000036ba       _cexit                     00000001800046ba f   ucrt:api-ms-win-crt-runtime-l1-1-0.dll
 0001:000036c0       __acrt_initialize          00000001800046c0 f   MSVCRT:ucrt_stubs.obj
 0001:000036c0       __acrt_thread_attach       00000001800046c0 f   MSVCRT:ucrt_stubs.obj
 0001:000036c0       __acrt_thread_detach       00000001800046c0 f   MSVCRT:ucrt_stubs.obj
 0001:000036c0       __acrt_uninitialize        00000001800046c0 f   MSVCRT:ucrt_stubs.obj
 0001:000036c0       __acrt_uninitialize_critical 00000001800046c0 f   MSVCRT:ucrt_stubs.obj
 0001:000036c0       __scrt_stub_for_acrt_initialize 00000001800046c0 f   MSVCRT:ucrt_stubs.obj
 0001:000036c0       __scrt_stub_for_acrt_thread_attach 00000001800046c0 f   MSVCRT:ucrt_stubs.obj
 0001:000036c0       __scrt_stub_for_acrt_thread_detach 00000001800046c0 f   MSVCRT:ucrt_stubs.obj
 0001:000036c0       __scrt_stub_for_acrt_uninitialize 00000001800046c0 f   MSVCRT:ucrt_stubs.obj
 0001:000036c0       __scrt_stub_for_acrt_uninitialize_critical 00000001800046c0 f   MSVCRT:ucrt_stubs.obj
 0001:000036c0       __vcrt_initialize          00000001800046c0 f   MSVCRT:ucrt_stubs.obj
 0001:000036c0       __vcrt_thread_attach       00000001800046c0 f   MSVCRT:ucrt_stubs.obj
 0001:000036c0       __vcrt_thread_detach       00000001800046c0 f   MSVCRT:ucrt_stubs.obj
 0001:000036c0       __vcrt_uninitialize        00000001800046c0 f   MSVCRT:ucrt_stubs.obj
 0001:000036c0       __vcrt_uninitialize_critical 00000001800046c0 f   MSVCRT:ucrt_stubs.obj
 0001:000036c4       __scrt_stub_for_is_c_termination_complete 00000001800046c4 f   MSVCRT:ucrt_stubs.obj
 0001:000036c4       _is_c_termination_complete 00000001800046c4 f   MSVCRT:ucrt_stubs.obj
 0001:000036e0       _guard_dispatch_icall_nop  00000001800046e0 f   MSVCRT:guard_dispatch.obj
 0001:00003700       _guard_xfg_dispatch_icall_nop 0000000180004700 f   MSVCRT:guard_xfg_dispatch.obj
 0002:00000000       __imp_RtlCaptureContext    0000000180005000     kernel32:KERNEL32.dll
 0002:00000008       __imp_RtlLookupFunctionEntry 0000000180005008     kernel32:KERNEL32.dll
 0002:00000010       __imp_RtlVirtualUnwind     0000000180005010     kernel32:KERNEL32.dll
 0002:00000018       __imp_UnhandledExceptionFilter 0000000180005018     kernel32:KERNEL32.dll
 0002:00000020       __imp_SetUnhandledExceptionFilter 0000000180005020     kernel32:KERNEL32.dll
 0002:00000028       __imp_GetCurrentProcess    0000000180005028     kernel32:KERNEL32.dll
 0002:00000030       __imp_TerminateProcess     0000000180005030     kernel32:KERNEL32.dll
 0002:00000038       __imp_IsProcessorFeaturePresent 0000000180005038     kernel32:KERNEL32.dll
 0002:00000040       __imp_CloseHandle          0000000180005040     kernel32:KERNEL32.dll
 0002:00000048       __imp_EnterCriticalSection 0000000180005048     kernel32:KERNEL32.dll
 0002:00000050       __imp_LeaveCriticalSection 0000000180005050     kernel32:KERNEL32.dll
 0002:00000058       __imp_InitializeCriticalSectionAndSpinCount 0000000180005058     kernel32:KERNEL32.dll
 0002:00000060       __imp_DeleteCriticalSection 0000000180005060     kernel32:KERNEL32.dll
 0002:00000068       __imp_SetEvent             0000000180005068     kernel32:KERNEL32.dll
 0002:00000070       __imp_ResetEvent           0000000180005070     kernel32:KERNEL32.dll
 0002:00000078       __imp_WaitForSingleObjectEx 0000000180005078     kernel32:KERNEL32.dll
 0002:00000080       __imp_CreateEventW         0000000180005080     kernel32:KERNEL32.dll
 0002:00000088       __imp_GetModuleHandleW     0000000180005088     kernel32:KERNEL32.dll
 0002:00000090       __imp_GetProcAddress       0000000180005090     kernel32:KERNEL32.dll
 0002:00000098       __imp_IsDebuggerPresent    0000000180005098     kernel32:KERNEL32.dll
 0002:000000a0       __imp_QueryPerformanceCounter 00000001800050a0     kernel32:KERNEL32.dll
 0002:000000a8       __imp_GetCurrentProcessId  00000001800050a8     kernel32:KERNEL32.dll
 0002:000000b0       __imp_GetCurrentThreadId   00000001800050b0     kernel32:KERNEL32.dll
 0002:000000b8       __imp_GetSystemTimeAsFileTime 00000001800050b8     kernel32:KERNEL32.dll
 0002:000000c0       __imp_DisableThreadLibraryCalls 00000001800050c0     kernel32:KERNEL32.dll
 0002:000000c8       __imp_InitializeSListHead  00000001800050c8     kernel32:KERNEL32.dll
 0002:000000d0       \177KERNEL32_NULL_THUNK_DATA 00000001800050d0     kernel32:KERNEL32.dll
 0002:000000d8       __imp_memcpy               00000001800050d8     vcruntime:VCRUNTIME140.dll
 0002:000000e0       __imp_memset               00000001800050e0     vcruntime:VCRUNTIME140.dll
 0002:000000e8       __imp_strchr               00000001800050e8     vcruntime:VCRUNTIME140.dll
 0002:000000f0       __imp___C_specific_handler 00000001800050f0     vcruntime:VCRUNTIME140.dll
 0002:000000f8       __imp___std_type_info_destroy_list 00000001800050f8     vcruntime:VCRUNTIME140.dll
 0002:00000100       \177VCRUNTIME140_NULL_THUNK_DATA 0000000180005100     vcruntime:VCRUNTIME140.dll
 0002:00000108       __imp__errno               0000000180005108     ucrt:api-ms-win-crt-runtime-l1-1-0.dll
 0002:00000110       __imp_exit                 0000000180005110     ucrt:api-ms-win-crt-runtime-l1-1-0.dll
 0002:00000118       __imp__cexit               0000000180005118     ucrt:api-ms-win-crt-runtime-l1-1-0.dll
 0002:00000120       __imp__crt_atexit          0000000180005120     ucrt:api-ms-win-crt-runtime-l1-1-0.dll
 0002:00000128       __imp__execute_onexit_table 0000000180005128     ucrt:api-ms-win-crt-runtime-l1-1-0.dll
 0002:00000130       __imp__register_onexit_function 0000000180005130     ucrt:api-ms-win-crt-runtime-l1-1-0.dll
 0002:00000138       __imp__initialize_onexit_table 0000000180005138     ucrt:api-ms-win-crt-runtime-l1-1-0.dll
 0002:00000140       __imp__initialize_narrow_environment 0000000180005140     ucrt:api-ms-win-crt-runtime-l1-1-0.dll
 0002:00000148       __imp__configure_narrow_argv 0000000180005148     ucrt:api-ms-win-crt-runtime-l1-1-0.dll
 0002:00000150       __imp__seh_filter_dll      0000000180005150     ucrt:api-ms-win-crt-runtime-l1-1-0.dll
 0002:00000158       __imp__initterm_e          0000000180005158     ucrt:api-ms-win-crt-runtime-l1-1-0.dll
 0002:00000160       __imp__initterm            0000000180005160     ucrt:api-ms-win-crt-runtime-l1-1-0.dll
 0002:00000168       \177api-ms-win-crt-runtime-l1-1-0_NULL_THUNK_DATA 0000000180005168     ucrt:api-ms-win-crt-runtime-l1-1-0.dll
 0002:00000170       __imp___acrt_iob_func      0000000180005170     ucrt:api-ms-win-crt-stdio-l1-1-0.dll
 0002:00000178       __imp_fflush               0000000180005178     ucrt:api-ms-win-crt-stdio-l1-1-0.dll
 0002:00000180       __imp___stdio_common_vsprintf 0000000180005180     ucrt:api-ms-win-crt-stdio-l1-1-0.dll
 0002:00000188       __imp___stdio_common_vfprintf 0000000180005188     ucrt:api-ms-win-crt-stdio-l1-1-0.dll
 0002:00000190       \177api-ms-win-crt-stdio-l1-1-0_NULL_THUNK_DATA 0000000180005190     ucrt:api-ms-win-crt-stdio-l1-1-0.dll
 0002:00000198       __imp__strdup              0000000180005198     ucrt:api-ms-win-crt-string-l1-1-0.dll
 0002:00000198       __imp_strdup               0000000180005198     ucrt:api-ms-win-crt-string-l1-1-0.dll
 0002:000001a0       __imp_strlen               00000001800051a0     ucrt:api-ms-win-crt-string-l1-1-0.dll
 0002:000001a8       __imp_strncpy              00000001800051a8     ucrt:api-ms-win-crt-string-l1-1-0.dll
 0002:000001b0       \177api-ms-win-crt-string-l1-1-0_NULL_THUNK_DATA 00000001800051b0     ucrt:api-ms-win-crt-string-l1-1-0.dll
 0002:000001b8       __guard_check_icall_fptr   00000001800051b8     MSVCRT:guard_support.obj
 0002:000001c0       __guard_xfg_check_icall_fptr 00000001800051c0     MSVCRT:guard_support.obj
 0002:000001c8       __guard_dispatch_icall_fptr 00000001800051c8     MSVCRT:guard_support.obj
 0002:000001d0       __guard_xfg_dispatch_icall_fptr 00000001800051d0     MSVCRT:guard_support.obj
 0002:000001d8       __guard_xfg_table_dispatch_icall_fptr 00000001800051d8     MSVCRT:guard_support.obj
 0002:000001e0       __castguard_check_failure_os_handled_fptr 00000001800051e0     MSVCRT:guard_support.obj
 0002:000001e8       __guard_memcpy_fptr        00000001800051e8     vcruntime:softmemtag.obj
 0002:000001f0       __xc_a                     00000001800051f0     MSVCRT:initializers.obj
 0002:000001f8       __xc_z                     00000001800051f8     MSVCRT:initializers.obj
 0002:00000200       __xi_a                     0000000180005200     MSVCRT:initializers.obj
 0002:00000210       __xi_z                     0000000180005210     MSVCRT:initializers.obj
 0002:00000218       __xl_a                     0000000180005218     MSVCRT:tlssup.obj
 0002:00000220       __xl_z                     0000000180005220     MSVCRT:tlssup.obj
 0002:00000228       __xp_a                     0000000180005228     MSVCRT:initializers.obj
 0002:00000230       __xp_z                     0000000180005230     MSVCRT:initializers.obj
 0002:00000238       __xt_a                     0000000180005238     MSVCRT:initializers.obj
 0002:00000240       __xt_z                     0000000180005240     MSVCRT:initializers.obj
 0002:00000250       g_refKindStr               0000000180005250     libpopframe004.obj
 0002:00000400       ??_C@_09BPLDFGCI@unknown_0@ 0000000180005400     libpopframe004.obj
 0002:00000410       ??_C@_0BL@FPNMECJD@JVMTI_HEAP_REFERENCE_CLASS@ 0000000180005410     libpopframe004.obj
 0002:00000430       ??_C@_0BL@FKGKKLNM@JVMTI_HEAP_REFERENCE_FIELD@ 0000000180005430     libpopframe004.obj
 0002:00000450       ??_C@_0CD@CAEHCFJF@JVMTI_HEAP_REFERENCE_ARRAY_ELEM@ 0000000180005450     libpopframe004.obj
 0002:00000478       ??_C@_0CC@DNEBMCNK@JVMTI_HEAP_REFERENCE_CLASS_LOAD@ 0000000180005478     libpopframe004.obj
 0002:000004a0       ??_C@_0BN@CJMIPEBB@JVMTI_HEAP_REFERENCE_SIGNERS@ 00000001800054a0     libpopframe004.obj
 0002:000004c0       ??_C@_0CH@HBOIDPEB@JVMTI_HEAP_REFERENCE_PROTECTION@ 00000001800054c0     libpopframe004.obj
 0002:000004e8       ??_C@_0BP@MDKGDGKL@JVMTI_HEAP_REFERENCE_INTERFACE@ 00000001800054e8     libpopframe004.obj
 0002:00000508       ??_C@_0CC@JJMIHNJH@JVMTI_HEAP_REFERENCE_STATIC_FIE@ 0000000180005508     libpopframe004.obj
 0002:00000530       ??_C@_0CD@IDHEEGID@JVMTI_HEAP_REFERENCE_CONSTANT_P@ 0000000180005530     libpopframe004.obj
 0002:00000558       ??_C@_0CA@EFFCHNG@JVMTI_HEAP_REFERENCE_SUPERCLASS@ 0000000180005558     libpopframe004.obj
 0002:00000578       ??_C@_0L@PCDFHGCJ@unknown_11@ 0000000180005578     libpopframe004.obj
 0002:00000588       ??_C@_0L@NJBICFOK@unknown_12@ 0000000180005588     libpopframe004.obj
 0002:00000598       ??_C@_0L@MAADBEKL@unknown_13@ 0000000180005598     libpopframe004.obj
 0002:000005a8       ??_C@_0L@IPECICGM@unknown_14@ 00000001800055a8     libpopframe004.obj
 0002:000005b8       ??_C@_0L@JGFJLDCN@unknown_15@ 00000001800055b8     libpopframe004.obj
 0002:000005c8       ??_C@_0L@LNHEOAOO@unknown_16@ 00000001800055c8     libpopframe004.obj
 0002:000005d8       ??_C@_0L@KEGPNBKP@unknown_17@ 00000001800055d8     libpopframe004.obj
 0002:000005e8       ??_C@_0L@CDPHMNGA@unknown_18@ 00000001800055e8     libpopframe004.obj
 0002:000005f8       ??_C@_0L@DKOMPMCB@unknown_19@ 00000001800055f8     libpopframe004.obj
 0002:00000608       ??_C@_0L@OJGIPJDB@unknown_20@ 0000000180005608     libpopframe004.obj
 0002:00000618       ??_C@_0CA@KAOFNDEM@JVMTI_HEAP_REFERENCE_JNI_GLOBAL@ 0000000180005618     libpopframe004.obj
 0002:00000638       ??_C@_0CC@HPFAJBK@JVMTI_HEAP_REFERENCE_SYSTEM_CLA@ 0000000180005638     libpopframe004.obj
 0002:00000660       ??_C@_0BN@FDEGFOHC@JVMTI_HEAP_REFERENCE_MONITOR@ 0000000180005660     libpopframe004.obj
 0002:00000680       ??_C@_0CB@HKIBCMAJ@JVMTI_HEAP_REFERENCE_STACK_LOCA@ 0000000180005680     libpopframe004.obj
 0002:000006a8       ??_C@_0BP@EAACMMOE@JVMTI_HEAP_REFERENCE_JNI_LOCAL@ 00000001800056a8     libpopframe004.obj
 0002:000006c8       ??_C@_0BM@IJDEOGOE@JVMTI_HEAP_REFERENCE_THREAD@ 00000001800056c8     libpopframe004.obj
 0002:000006e8       ??_C@_0BL@EDGPPKC@JVMTI_HEAP_REFERENCE_OTHER@ 00000001800056e8     libpopframe004.obj
 0002:00000704       ??_C@_04BCJPDBDA@Code@     0000000180005704     libpopframe004.obj
 0002:00000710       ??_C@_0BA@OCLMCFKC@LineNumberTable@ 0000000180005710     libpopframe004.obj
 0002:00000720       ??_C@_0BD@CPAEPILC@LocalVariableTable@ 0000000180005720     libpopframe004.obj
 0002:00000738       ??_C@_0BH@NMBDNHBD@LocalVariableTypeTable@ 0000000180005738     libpopframe004.obj
 0002:00000750       ??_C@_0O@HIHEEDNJ@StackMapTable@ 0000000180005750     libpopframe004.obj
 0002:00000760       ??_C@_0L@HCDIAMJG@?9?5?$CFs?0?5?$CFd?3?5@ 0000000180005760     libpopframe004.obj
 0002:00000770       ??_C@_0JI@HLPECLFI@?$CD?5?4?4?4?6?$CD?5ERROR?3?5too?5many?5complai@ 0000000180005770     libpopframe004.obj
 0002:00000810       ??_C@_0ED@JNEKCCOB@The?5following?5fake?5exception?5st@ 0000000180005810     libpopframe004.obj
 0002:00000858       ??_C@_0CN@FCNMDFBH@nsk?4share?4Fake_Exception_for_RU@ 0000000180005858     libpopframe004.obj
 0002:00000888       ??_C@_08PGFFNAEI@?$CI?$CFs?3?$CFd?$CJ?5@ 0000000180005888     libpopframe004.obj
 0002:00000898       ??_C@_0DP@IENMAEGI@s?2test?2hotspot?2jtreg?2vmTestbase@ 0000000180005898     libpopframe004.obj
 0002:000008d8       ??_C@_0BL@NDJLFFJB@?7at?5nsk_lvcomplain?$CI?$CFs?3?$CFd?$CJ?6@ 00000001800058d8     libpopframe004.obj
 0002:000008f8       ??_C@_0BC@JOOKAFKF@?$CD?5ERROR?3?5?$CFs?0?5?$CFd?3?5@ 00000001800058f8     libpopframe004.obj
 0002:00000910       ??_C@_09KJEAHMEH@?$CD?5ERROR?3?5@ 0000000180005910     libpopframe004.obj
 0002:0000091c       ??_C@_02GPIOPFAK@?$DO?$DO@ 000000018000591c     libpopframe004.obj
 0002:00000920       ??_C@_02FODMEDOG@?$DM?$DM@ 0000000180005920     libpopframe004.obj
 0002:00000924       ??_C@_02DJGKEECL@?4?4@     0000000180005924     libpopframe004.obj
 0002:00000928       ??_C@_0O@CJPGJOAF@?9?5?$CFs?0?5?$CFd?3?5?$CFs?5@ 0000000180005928     libpopframe004.obj
 0002:00000938       ??_C@_0CB@IAKPDOIC@?$CD?5?5?5verified?5assertion?5is?5FALSE@ 0000000180005938     libpopframe004.obj
 0002:00000960       ??_C@_0CO@LGONDEPD@stdout?3?5fflush?5failed?5?9?5err?$DN?$CFd?5@ 0000000180005960     libpopframe004.obj
 0002:00000990       ??_C@_0CO@KBGKJPBD@stderr?3?5fflush?5failed?5?9?5err?$DN?$CFd?5@ 0000000180005990     libpopframe004.obj
 0002:000009c0       ??_C@_0DM@KLJPMIDM@check_jvmti_status?3?5JVMTI?5funct@ 00000001800059c0     libpopframe004.obj
 0002:00000a00       ??_C@_0CL@MEELKAEL@deallocate?3?5error?5in?5JVMTI?5Deal@ 0000000180005a00     libpopframe004.obj
 0002:00000a30       ??_C@_0DO@CNKPCOHC@get_method_class_name?3?5error?5in@ 0000000180005a30     libpopframe004.obj
 0002:00000a70       ??_C@_0DI@ODOBMANA@get_method_class_name?3?5error?5in@ 0000000180005a70     libpopframe004.obj
 0002:00000aa8       ??_C@_0CP@IBPBEBM@get_method_class_name?3?5error?5in@ 0000000180005aa8     libpopframe004.obj
 0002:00000ad8       ??_C@_0CL@BDMIAND@print_method?3?5error?5in?5JVMTI?5Ge@ 0000000180005ad8     libpopframe004.obj
 0002:00000b08       ??_C@_0P@GFDDDNG@?$CF2d?3?5?$CFs?3?5?$CFs?$CFs?6@ 0000000180005b08     libpopframe004.obj
 0002:00000b18       ??_C@_01EEMJAFIK@?6@       0000000180005b18     libpopframe004.obj
 0002:00000b20       ??_C@_0BB@NEONAMMP@?$DMUnnamed?5thread?$DO@ 0000000180005b20     libpopframe004.obj
 0002:00000b38       ??_C@_0DD@PEIMAGBL@get_thread_name?3?5error?5in?5JVMTI@ 0000000180005b38     libpopframe004.obj
 0002:00000b70       ??_C@_0DA@DGJBBBMN@print_stack_trace?3?5error?5in?5JVM@ 0000000180005b70     libpopframe004.obj
 0002:00000ba0       ??_C@_0DC@EJGPEKOE@JVMTI?5Stack?5Trace?5for?5thread?5?$CFs@ 0000000180005ba0     libpopframe004.obj
 0002:00000bd8       ??_C@_0BB@JCNMKLLK@JVMTI_ERROR_NONE@ 0000000180005bd8     libpopframe004.obj
 0002:00000bf0       ??_C@_0BL@LDIMKLPH@JVMTI_ERROR_INVALID_THREAD@ 0000000180005bf0     libpopframe004.obj
 0002:00000c10       ??_C@_0CB@PJFPAIKJ@JVMTI_ERROR_INVALID_THREAD_GROU@ 0000000180005c10     libpopframe004.obj
 0002:00000c38       ??_C@_0BN@LLMKHMNF@JVMTI_ERROR_INVALID_PRIORITY@ 0000000180005c38     libpopframe004.obj
 0002:00000c58       ??_C@_0CB@MBOFKAGB@JVMTI_ERROR_THREAD_NOT_SUSPENDE@ 0000000180005c58     libpopframe004.obj
 0002:00000c80       ??_C@_0BN@FABOLPBI@JVMTI_ERROR_THREAD_SUSPENDED@ 0000000180005c80     libpopframe004.obj
 0002:00000ca0       ??_C@_0BN@FDGNOBJM@JVMTI_ERROR_THREAD_NOT_ALIVE@ 0000000180005ca0     libpopframe004.obj
 0002:00000cc0       ??_C@_0BL@GOBIFKNJ@JVMTI_ERROR_INVALID_OBJECT@ 0000000180005cc0     libpopframe004.obj
 0002:00000ce0       ??_C@_0BK@FCMAJPPC@JVMTI_ERROR_INVALID_CLASS@ 0000000180005ce0     libpopframe004.obj
 0002:00000d00       ??_C@_0BP@IKLLBKEB@JVMTI_ERROR_CLASS_NOT_PREPARED@ 0000000180005d00     libpopframe004.obj
 0002:00000d20       ??_C@_0BN@KLPPLKG@JVMTI_ERROR_INVALID_METHODID@ 0000000180005d20     libpopframe004.obj
 0002:00000d40       ??_C@_0BN@BCEKOKND@JVMTI_ERROR_INVALID_LOCATION@ 0000000180005d40     libpopframe004.obj
 0002:00000d60       ??_C@_0BM@DFDGPME@JVMTI_ERROR_INVALID_FIELDID@ 0000000180005d60     libpopframe004.obj
 0002:00000d80       ??_C@_0BL@NELIEPEC@JVMTI_ERROR_NO_MORE_FRAMES@ 0000000180005d80     libpopframe004.obj
 0002:00000da0       ??_C@_0BJ@BDBECFDM@JVMTI_ERROR_OPAQUE_FRAME@ 0000000180005da0     libpopframe004.obj
 0002:00000dc0       ??_C@_0BK@MIIFNLOB@JVMTI_ERROR_TYPE_MISMATCH@ 0000000180005dc0     libpopframe004.obj
 0002:00000de0       ??_C@_0BJ@HPCAOILC@JVMTI_ERROR_INVALID_SLOT@ 0000000180005de0     libpopframe004.obj
 0002:00000e00       ??_C@_0BG@CHILOPNI@JVMTI_ERROR_DUPLICATE@ 0000000180005e00     libpopframe004.obj
 0002:00000e18       ??_C@_0BG@DIEMLHKM@JVMTI_ERROR_NOT_FOUND@ 0000000180005e18     libpopframe004.obj
 0002:00000e30       ??_C@_0BM@NHMCKHOB@JVMTI_ERROR_INVALID_MONITOR@ 0000000180005e30     libpopframe004.obj
 0002:00000e50       ??_C@_0BO@PPEDAJGL@JVMTI_ERROR_NOT_MONITOR_OWNER@ 0000000180005e50     libpopframe004.obj
 0002:00000e70       ??_C@_0BG@FCAIPEID@JVMTI_ERROR_INTERRUPT@ 0000000180005e70     libpopframe004.obj
 0002:00000e88       ??_C@_0CB@EGDBNKOI@JVMTI_ERROR_INVALID_CLASS_FORMA@ 0000000180005e88     libpopframe004.obj
 0002:00000eb0       ??_C@_0CG@DGKOGIAL@JVMTI_ERROR_CIRCULAR_CLASS_DEFI@ 0000000180005eb0     libpopframe004.obj
 0002:00000ed8       ??_C@_0BP@ICEALPKC@JVMTI_ERROR_FAILS_VERIFICATION@ 0000000180005ed8     libpopframe004.obj
 0002:00000ef8       ??_C@_0DC@JDACLMIO@JVMTI_ERROR_UNSUPPORTED_REDEFIN@ 0000000180005ef8     libpopframe004.obj
 0002:00000f30       ??_C@_0DE@GKDKNOMJ@JVMTI_ERROR_UNSUPPORTED_REDEFIN@ 0000000180005f30     libpopframe004.obj
 0002:00000f68       ??_C@_0BO@LAFKIOG@JVMTI_ERROR_INVALID_TYPESTATE@ 0000000180005f68     libpopframe004.obj
 0002:00000f88       ??_C@_0DH@INDGCLLB@JVMTI_ERROR_UNSUPPORTED_REDEFIN@ 0000000180005f88     libpopframe004.obj
 0002:00000fc0       ??_C@_0DE@NHEOMMGI@JVMTI_ERROR_UNSUPPORTED_REDEFIN@ 0000000180005fc0     libpopframe004.obj
 0002:00000ff8       ??_C@_0CA@EKPNJOEP@JVMTI_ERROR_UNSUPPORTED_VERSION@ 0000000180005ff8     libpopframe004.obj
 0002:00001018       ??_C@_0BN@OFFMAHHL@JVMTI_ERROR_NAMES_DONT_MATCH@ 0000000180006018     libpopframe004.obj
 0002:00001038       ??_C@_0DN@HHBBLAKE@JVMTI_ERROR_UNSUPPORTED_REDEFIN@ 0000000180006038     libpopframe004.obj
 0002:00001078       ??_C@_0DO@HMBGBGNA@JVMTI_ERROR_UNSUPPORTED_REDEFIN@ 0000000180006078     libpopframe004.obj
 0002:000010b8       ??_C@_0BP@PBECGKHJ@JVMTI_ERROR_UNMODIFIABLE_CLASS@ 00000001800060b8     libpopframe004.obj
 0002:000010d8       ??_C@_0BK@CANILEHF@JVMTI_ERROR_NOT_AVAILABLE@ 00000001800060d8     libpopframe004.obj
 0002:000010f8       ??_C@_0CE@INJKMEFK@JVMTI_ERROR_MUST_POSSESS_CAPABI@ 00000001800060f8     libpopframe004.obj
 0002:00001120       ??_C@_0BJ@LBFPFPDM@JVMTI_ERROR_NULL_POINTER@ 0000000180006120     libpopframe004.obj
 0002:00001140       ??_C@_0BP@CHJPNNEM@JVMTI_ERROR_ABSENT_INFORMATION@ 0000000180006140     libpopframe004.obj
 0002:00001160       ??_C@_0BP@OMFMNLC@JVMTI_ERROR_INVALID_EVENT_TYPE@ 0000000180006160     libpopframe004.obj
 0002:00001180       ??_C@_0BN@BIBNPHHO@JVMTI_ERROR_ILLEGAL_ARGUMENT@ 0000000180006180     libpopframe004.obj
 0002:000011a0       ??_C@_0BK@KKNDHDCE@JVMTI_ERROR_NATIVE_METHOD@ 00000001800061a0     libpopframe004.obj
 0002:000011c0       ??_C@_0BK@PMKCFHAE@JVMTI_ERROR_OUT_OF_MEMORY@ 00000001800061c0     libpopframe004.obj
 0002:000011e0       ??_C@_0BK@NNJBDMNB@JVMTI_ERROR_ACCESS_DENIED@ 00000001800061e0     libpopframe004.obj
 0002:00001200       ??_C@_0BI@GHECLMNC@JVMTI_ERROR_WRONG_PHASE@ 0000000180006200     libpopframe004.obj
 0002:00001218       ??_C@_0BF@OLIHJOII@JVMTI_ERROR_INTERNAL@ 0000000180006218     libpopframe004.obj
 0002:00001230       ??_C@_0BO@EOHGKJHI@JVMTI_ERROR_UNATTACHED_THREAD@ 0000000180006230     libpopframe004.obj
 0002:00001250       ??_C@_0CA@LKHFDACL@JVMTI_ERROR_INVALID_ENVIRONMENT@ 0000000180006250     libpopframe004.obj
 0002:00001270       ??_C@_0BA@MMFHLOKK@?$DMunknown?5error?$DO@ 0000000180006270     libpopframe004.obj
 0002:00001280       ??_C@_0CF@CBHOKDB@throwable?5?$DN?5jni?9?$DOExceptionOccur@ 0000000180006280     libpopframe004.obj
 0002:000012a8       ??_C@_03OFAPEBGM@?$CFs?6@  00000001800062a8     libpopframe004.obj
 0002:000012b0       ??_C@_0DM@LPIGEGNJ@s?2test?2hotspot?2jtreg?2vmTestbase@ 00000001800062b0     libpopframe004.obj
 0002:000012f0       ??_C@_0CC@NFCNPEPK@Exception?5in?5JNI?5call?5?$CIcleared?$CJ@ 00000001800062f0     libpopframe004.obj
 0002:00001318       ??_C@_0BJ@IBAKFIKF@jni?9?$DOExceptionDescribe?$CI?$CJ@ 0000000180006318     libpopframe004.obj
 0002:00001338       ??_C@_0BG@GGKALKMH@jni?9?$DOExceptionClear?$CI?$CJ@ 0000000180006338     libpopframe004.obj
 0002:00001350       ??_C@_0CF@JMGFGJLJ@?$CD?5?5?5verified?5JNI?5assertion?5is?5F@ 0000000180006350     libpopframe004.obj
 0002:00001378       ??_C@_0CB@MLNJNCLJ@?5?5jvmti?5error?3?5code?$DN?$CFd?0?5name?$DN?$CFs@ 0000000180006378     libpopframe004.obj
 0002:000013a0       ??_C@_0CD@OHBGDKMK@?$CD?5?5?5jvmti?5error?3?5code?$DN?$CFd?0?5name?$DN@ 00000001800063a0     libpopframe004.obj
 0002:000013c8       ??_C@_0CG@JNNCGPHB@?$CD?5?5?5error?5expected?3?5code?$DN?$CFd?0?5na@ 00000001800063c8     libpopframe004.obj
 0002:000013f0       ??_C@_0EB@IMGKPCGE@?$CIstr_obj?5?$DN?5jni?9?$DONewStringUTF?$CIco@ 00000001800063f0     libpopframe004.obj
 0002:00001440       ??_C@_0EA@HFOGGBCC@s?2test?2hotspot?2jtreg?2vmTestbase@ 0000000180006440     libpopframe004.obj
 0002:00001480       ??_C@_0CB@PKFNCBLK@?$DO?$DO?$DO?$DO?$DO?$DO?$DO?$DO?5Invoke?5SuspendThread?$CI?$CJ@ 0000000180006480     libpopframe004.obj
 0002:000014a8       ??_C@_0DC@FMKOEGFG@?$CFs?3?5Failed?5to?5call?5SuspendThrea@ 00000001800064a8     libpopframe004.obj
 0002:000014e0       ??_C@_0CP@PCCFKDM@?$DM?$DM?$DM?$DM?$DM?$DM?$DM?$DM?5SuspendThread?$CI?$CJ?5is?5suc@ 00000001800064e0     libpopframe004.obj
 0002:00001510       ??_C@_05KKCIMGE@error@     0000000180006510     libpopframe004.obj
 0002:00001518       ??_C@_0CJ@JACLEAA@Test?5failed?5by?5setFailStatus?$CI?$CJ?4@ 0000000180006518     libpopframe004.obj
 0002:00001550       ??_C@_0EA@PNBCDMOA@s?2test?2hotspot?2jtreg?2vmTestbase@ 0000000180006550     libpopframe004.obj
 0002:00001590       ??_C@_0DI@ILAHDLMP@?$CI?$CKagentThreadProc?$CJ?$CIjvmti_env?0?5a@ 0000000180006590     libpopframe004.obj
 0002:000015c8       ??_C@_0BD@KDBALNLB@JVMTI?5agent?5thread@ 00000001800065c8     libpopframe004.obj
 0002:000015e0       ??_C@_0BB@NOKBFPFO@java?1lang?1Thread@ 00000001800065e0     libpopframe004.obj
 0002:000015f4       ??_C@_06FALKBLGB@?$DMinit?$DO@ 00000001800065f4     libpopframe004.obj
 0002:00001600       ??_C@_0BG@IKDDPPGD@?$CILjava?1lang?1String?$DL?$CJV@ 0000000180006600     libpopframe004.obj
 0002:00001620       ??_C@_0EB@IFJBFEKC@?$CIthreadClass?5?$DN?5jni_env?9?$DOFindCla@ 0000000180006620     libpopframe004.obj
 0002:00001670       ??_C@_0GF@FGFIBKKL@?$CIthreadCtor?5?$DN?5jni_env?9?$DOGetMetho@ 0000000180006670     libpopframe004.obj
 0002:000016d8       ??_C@_0DN@NCPDJLOG@?$CIthreadName?5?$DN?5jni_env?9?$DONewStrin@ 00000001800066d8     libpopframe004.obj
 0002:00001720       ??_C@_0FE@PFKODBGC@?$CIthreadObject?5?$DN?5jni_env?9?$DONewObj@ 0000000180006720     libpopframe004.obj
 0002:00001780       ??_C@_0ED@HOBAHHJI@?$CIthreadGlobalRef?5?$DN?5jni_env?9?$DONew@ 0000000180006780     libpopframe004.obj
 0002:000017d0       ??_C@_0FN@HNJJAHFC@jvmti_env?9?$DORunAgentThread?$CIagent@ 00000001800067d0     libpopframe004.obj
 0002:00001830       ??_C@_0EA@MOJDNKDF@Debuggee?5status?5sync?5aborted?5be@ 0000000180006830     libpopframe004.obj
 0002:00001870       ??_C@_0EA@EEOEJAEN@status?5?$DN?5syncDebuggeeStatus?$CIjni@ 0000000180006870     libpopframe004.obj
 0002:000018b0       ??_C@_0BL@JBCFNBMB@nsk_jvmti_resetAgentData?$CI?$CJ@ 00000001800068b0     libpopframe004.obj
 0002:000018d0       ??_C@_0EL@LPBEELIP@s?2test?2hotspot?2jtreg?2vmTestbase@ 00000001800068d0     libpopframe004.obj
 0002:00001920       ??_C@_0CK@JDAMFDMJ@jvmti?9?$DOSetTag?$CIo?0?5tag?$CJ?5?$DN?$DN?5JVMTI_@ 0000000180006920     libpopframe004.obj
 0002:00001950       ??_C@_0CC@DAMNHKNI@Can?8t?5set?5tag?5?$CFli?5for?5object?5?$CFl@ 0000000180006950     libpopframe004.obj
 0002:00001978       ??_C@_0DL@HAJPNKEF@jvmti?9?$DOGetObjectHashCode?$CIo?0?5?$CGha@ 0000000180006978     libpopframe004.obj
 0002:000019b8       ??_C@_0BL@JFPIEOBF@Can?8t?5get?5hash?5object?5?$CFlx?6@ 00000001800069b8     libpopframe004.obj
 0002:000019d8       ??_C@_0BG@DICPHBKN@setTag?3?5?$CF08x?5?$DM?9?5?$CF?53li@ 00000001800069d8     libpopframe004.obj
 0002:000019f0       ??_C@_0DH@FCEEBDMJ@?$CIs?5?$DN?5jni?9?$DOGetStringUTFChars?$CIsIn@ 00000001800069f0     libpopframe004.obj
 0002:00001a28       ??_C@_0BJ@OKKGHDCN@Can?8t?5get?5string?5at?5?$CF?$CDp?6@ 0000000180006a28     libpopframe004.obj
 0002:00001a48       ??_C@_0BP@EKFLGGFJ@Can?8t?5get?5string?5at?5?$CF?$CDp?3?5null?6@ 0000000180006a48     libpopframe004.obj
 0002:00001a68       ??_C@_06ICODBHCL@?5?1?1?5?$CFs@ 0000000180006a68     libpopframe004.obj
 0002:00001a70       ??_C@_0DB@KGFPLEGO@?$CIr?5?$DN?5jvmti?9?$DOGetTag?$CIo?0?5?$CGtag?$CJ?$CJ?5?$DN?$DN@ 0000000180006a70     libpopframe004.obj
 0002:00001aa8       ??_C@_0CO@PDAGBCGJ@Can?8t?5GetTag?5for?5object?5?$CFlx?4?5Re@ 0000000180006aa8     libpopframe004.obj
 0002:00001ad8       ??_C@_0CH@HPEODOHC@TEST_BUG?3?5Max?4?5number?5of?5refs?5r@ 0000000180006ad8     libpopframe004.obj
 0002:00001b00       ??_C@_0DI@PHFCABIM@?$CIr?5?$DN?5jvmti?9?$DOGetTag?$CIfrom?0?5?$CGtagFr@ 0000000180006b00     libpopframe004.obj
 0002:00001b38       ??_C@_0DI@MDEGFNKD@TEST_BUG?3?5Can?8t?5GetTag?5for?5obje@ 0000000180006b38     libpopframe004.obj
 0002:00001b70       ??_C@_0DE@MLELJAHM@?$CIr?5?$DN?5jvmti?9?$DOGetTag?$CIto?0?5?$CGtagTo?$CJ?$CJ@ 0000000180006b70     libpopframe004.obj
 0002:00001ba4       ??_C@_03GAEACAIP@?$CI?$CJV@ 0000000180006ba4     libpopframe004.obj
 0002:00001ba8       ??_C@_0CD@GAGNNEOH@?$CD?$CD?$CD?$CD?5FramePop?5event?5occurred?5?$CD?$CD@ 0000000180006ba8     libpopframe004.obj
 0002:00001bd0       ??_C@_0CF@CKNHIJHL@?$CD?$CD?$CD?$CD?5MethodExit?5event?5occurred?5@ 0000000180006bd0     libpopframe004.obj
 0002:00001c00       ??_C@_0EP@HBCKCKG@s?2test?2hotspot?2jtreg?2vmTestbase@ 0000000180006c00     libpopframe004.obj
 0002:00001c50       ??_C@_0CA@LCONHFJP@?$DO?$DO?$DO?$DO?$DO?$DO?$DO?$DO?5Invoke?5ResumeThread?$CI?$CJ?6@ 0000000180006c50     libpopframe004.obj
 0002:00001c70       ??_C@_0DB@GNNPBNHM@?$CFs?3?5Failed?5to?5call?5ResumeThread@ 0000000180006c70     libpopframe004.obj
 0002:00001ca8       ??_C@_0CO@ONBIKMHM@?$DM?$DM?$DM?$DM?$DM?$DM?$DM?$DM?5ResumeThread?$CI?$CJ?5is?5succ@ 0000000180006ca8     libpopframe004.obj
 0002:00001cd8       ??_C@_0CN@GHJIKGLO@Failed?5to?5enable?5METHOD_EXIT?5ev@ 0000000180006cd8     libpopframe004.obj
 0002:00001d08       ??_C@_0CL@EPIEADBE@Failed?5to?5enable?5FRAME_POP?5even@ 0000000180006d08     libpopframe004.obj
 0002:00001d38       ??_C@_0BM@MACMONCJ@?$DO?$DO?$DO?$DO?$DO?$DO?$DO?$DO?5Invoke?5PopFrame?$CI?$CJ?6@ 0000000180006d38     libpopframe004.obj
 0002:00001d58       ??_C@_0DA@JCHFBMJO@Check?5FAILED?3?5PopFrame?$CI?$CJ?5was?5un@ 0000000180006d58     libpopframe004.obj
 0002:00001d88       ??_C@_0DJ@OIJKEFDI@Check?5PASSED?3?5PopFrame?$CI?$CJ?5failed@ 0000000180006d88     libpopframe004.obj
 0002:00001dc8       ??_C@_0DL@EFCJGIDB@Check?5FAILED?3?5PopFrame?$CI?$CJ?5return@ 0000000180006dc8     libpopframe004.obj
 0002:00001e10       ??_C@_0EB@CHLIAMDM@?7For?5more?5info?5about?5this?5error@ 0000000180006e10     libpopframe004.obj
 0002:00001e60       ??_C@_0EI@KHFEBDGK@TEST?5FAILED?3?5?$CFd?5JVMTI?5events?5we@ 0000000180006e60     libpopframe004.obj
 0002:00001eb0       ??_C@_0EJ@HNFLGOBM@Check?5PASSED?3?5No?5JVMTI?5events?5w@ 0000000180006eb0     libpopframe004.obj
 0002:00001f00       ??_C@_0CJ@KCDEKOCJ@Wrong?5result?5of?5a?5valid?5call?5to@ 0000000180006f00     libpopframe004.obj
 0002:00001f30       ??_C@_0DG@LAJPGIIE@?$CIGetPotentialCapabilities?$CJ?5unex@ 0000000180006f30     libpopframe004.obj
 0002:00001f68       ??_C@_0CN@LKPEOJPO@?$CIAddCapabilities?$CJ?5unexpected?5er@ 0000000180006f68     libpopframe004.obj
 0002:00001f98       ??_C@_0CN@BCCBOHCH@?$CIGetCapabilities?$CJ?5unexpected?5er@ 0000000180006f98     libpopframe004.obj
 0002:00001fc8       ??_C@_0CG@MCCDAOGE@Warning?3?5PopFrame?5is?5not?5implem@ 0000000180006fc8     libpopframe004.obj
 0002:00001ff0       ??_C@_0CM@FEKJDMLD@Warning?3?5suspend?1resume?5is?5not?5@ 0000000180006ff0     libpopframe004.obj
 0002:00002020       ??_C@_0CP@IMINGNLL@?$CISetEventCallbacks?$CJ?5unexpected?5@ 0000000180007020     libpopframe004.obj
 0002:00002050       ??_C@_0DK@CDIPDFNJ@Warning?3?5FramePop?5or?5MethodExit@ 0000000180007050     libpopframe004.obj
 0002:00002090       ??_C@_0BB@NOLAGKMP@watch_ev_monitor@ 0000000180007090     libpopframe004.obj
 0002:000020a8       ??_C@_0CO@BLGNGBDG@?$CICreateRawMonitor?$CJ?5unexpected?5e@ 00000001800070a8     libpopframe004.obj
 0002:000020d8       ??_C@_0N@MJKGCPBI@activeMethod@ 00000001800070d8     libpopframe004.obj
 0002:000020e8       ??_C@_0DG@OEHIFCJN@TEST?5FAILURE?3?5nativeMeth2?$CI?$CJ?3?5Un@ 00000001800070e8     libpopframe004.obj
 0002:00002120       ??_C@_0DA@NJEGGOM@nativeMeth2?$CI?$CJ?3?5calling?5the?5Java@ 0000000180007120     libpopframe004.obj
 0002:00002150       ??_C@_0DA@BMOIJHIH@nativeMeth?$CI?$CJ?3?5calling?5the?5nativ@ 0000000180007150     libpopframe004.obj
 0002:00002190       ??_C@_1EC@JIJBPKFM@?$AAa?$AAp?$AAi?$AA?9?$AAm?$AAs?$AA?9?$AAw?$AAi?$AAn?$AA?9?$AAc?$AAo?$AAr?$AAe@ 0000000180007190     MSVCRT:thread_safe_statics.obj
 0002:000021d8       ??_C@_1BK@MGMFAEKH@?$AAk?$AAe?$AAr?$AAn?$AAe?$AAl?$AA3?$AA2?$AA?4?$AAd?$AAl?$AAl@ 00000001800071d8     MSVCRT:thread_safe_statics.obj
 0002:000021f8       ??_C@_0BJ@JEBJOJFJ@SleepConditionVariableCS@ 00000001800071f8     MSVCRT:thread_safe_statics.obj
 0002:00002218       ??_C@_0BJ@PGPPEPCC@WakeAllConditionVariable@ 0000000180007218     MSVCRT:thread_safe_statics.obj
 0002:00002238       _pDefaultRawDllMain        0000000180007238     MSVCRT:dll_dllmain.obj
 0002:00002238       _pRawDllMain               0000000180007238     MSVCRT:dll_dllmain.obj
 0002:00002240       __xmm@ffffffffffffffffffffffffffffffff 0000000180007240     MSVCRT:utility.obj
 0002:00002250       _load_config_used          0000000180007250     MSVCRT:loadcfg.obj
 0002:00002400       _tls_used                  0000000180007400     MSVCRT:tlssup.obj
 0002:00002428       __volatile_metadata        0000000180007428     <linker-defined>
 0002:000027e8       __rtc_iaa                  00000001800077e8     MSVCRT:initsect.obj
 0002:000027f0       __rtc_izz                  00000001800077f0     MSVCRT:initsect.obj
 0002:000027f8       __rtc_taa                  00000001800077f8     MSVCRT:initsect.obj
 0002:00002800       __rtc_tzz                  0000000180007800     MSVCRT:initsect.obj
 0002:00002808       _tls_start                 0000000180007808     MSVCRT:tlssup.obj
 0002:0000280c       _Init_thread_epoch         000000018000780c     MSVCRT:thread_safe_statics.obj
 0002:00002810       _tls_end                   0000000180007810     MSVCRT:tlssup.obj
 0002:00002f60       __IMPORT_DESCRIPTOR_KERNEL32 0000000180007f60     kernel32:KERNEL32.dll
 0002:00002f74       __IMPORT_DESCRIPTOR_VCRUNTIME140 0000000180007f74     vcruntime:VCRUNTIME140.dll
 0002:00002f88       __IMPORT_DESCRIPTOR_api-ms-win-crt-runtime-l1-1-0 0000000180007f88     ucrt:api-ms-win-crt-runtime-l1-1-0.dll
 0002:00002f9c       __IMPORT_DESCRIPTOR_api-ms-win-crt-stdio-l1-1-0 0000000180007f9c     ucrt:api-ms-win-crt-stdio-l1-1-0.dll
 0002:00002fb0       __IMPORT_DESCRIPTOR_api-ms-win-crt-string-l1-1-0 0000000180007fb0     ucrt:api-ms-win-crt-string-l1-1-0.dll
 0002:00002fc4       __NULL_IMPORT_DESCRIPTOR   0000000180007fc4     kernel32:KERNEL32.dll
 0003:00000038       _Init_global_epoch         0000000180009038     MSVCRT:thread_safe_statics.obj
 0003:00000040       __security_cookie          0000000180009040     MSVCRT:gs_cookie.obj
 0003:00000048       __security_cookie_complement 0000000180009048     MSVCRT:gs_cookie.obj
 0003:00000050       __scrt_native_dllmain_reason 0000000180009050     MSVCRT:utility.obj
 0003:00000058       __isa_available            0000000180009058     MSVCRT:cpu_disp.obj
 0003:0000005c       __isa_enabled              000000018000905c     MSVCRT:cpu_disp.obj
 0003:00000060       __memset_fast_string_threshold 0000000180009060     MSVCRT:cpu_disp.obj
 0003:00000068       __memset_nt_threshold      0000000180009068     MSVCRT:cpu_disp.obj
 0003:00000070       __scrt_ucrt_dll_is_in_use  0000000180009070     MSVCRT:ucrt_stubs.obj
 0003:00000080       g_wrongHeapCallbacks       0000000180009080     libpopframe004.obj
 0003:00000100       g_szTagInfo                0000000180009100     libpopframe004.obj
 0003:00002040       g_tagFlags                 000000018000b040     libpopframe004.obj
 0003:00002428       g_refsToVerifyCnt          000000018000b428     libpopframe004.obj
 0003:0000242c       g_fakeUserData             000000018000b42c     libpopframe004.obj
 0003:00002430       g_tagVisitCount            000000018000b430     libpopframe004.obj
 0003:000033d0       g_refsToVerify             000000018000c3d0     libpopframe004.obj
 0003:0001aad0       g_userDataError            0000000180023ad0     libpopframe004.obj
 0003:0001add0       ?_OptionsStorage@?1??__local_stdio_printf_options@@9@4_KA 0000000180023dd0     libpopframe004.obj
 0003:0001b3a8       _tls_index                 00000001800243a8     MSVCRT:tlssup.obj
 0003:0001b3b0       __scrt_current_native_startup_state 00000001800243b0     MSVCRT:utility.obj
 0003:0001b3b8       __scrt_native_startup_lock 00000001800243b8     MSVCRT:utility.obj
 0003:0001b3f8       __scrt_debugger_hook_flag  00000001800243f8     MSVCRT:utility_desktop.obj
 0003:0001b400       ?__type_info_root_node@@3U__type_info_node@@A 0000000180024400     MSVCRT:tncleanup.obj
 0003:0001b410       ?_OptionsStorage@?1??__local_stdio_scanf_options@@9@4_KA 0000000180024410     MSVCRT:default_local_stdio_options.obj
 0003:0001b418       __favor                    0000000180024418     MSVCRT:cpu_disp.obj
 0003:0001b420       __dyn_tls_init_callback    0000000180024420     <common>

 entry point at        0001:00002df0

 Static symbols

 0000:fffd9000       .debug$S                   0000000180000000     popframe004.exp
 0000:fffd9000       .debug$S                   0000000180000000     vcruntime:VCRUNTIME140.dll
 0000:fffd9000       .debug$S                   0000000180000000     vcruntime:VCRUNTIME140.dll
 0000:fffd9000       .debug$S                   0000000180000000     vcruntime:VCRUNTIME140.dll
 0000:fffd9000       .debug$S                   0000000180000000     vcruntime:VCRUNTIME140.dll
 0000:fffd9000       .debug$S                   0000000180000000     vcruntime:VCRUNTIME140.dll
 0000:fffd9000       .debug$S                   0000000180000000     vcruntime:VCRUNTIME140.dll
 0000:fffd9000       .debug$S                   0000000180000000     vcruntime:VCRUNTIME140.dll
 0000:fffd9000       .debug$S                   0000000180000000     ucrt:api-ms-win-crt-convert-l1-1-0.dll
 0002:ffffb000       .idata$6                   0000000180000000     ucrt:api-ms-win-crt-convert-l1-1-0.dll
 0000:fffd9000       .debug$S                   0000000180000000     ucrt:api-ms-win-crt-heap-l1-1-0.dll
 0000:fffd9000       .debug$S                   0000000180000000     ucrt:api-ms-win-crt-heap-l1-1-0.dll
 0000:fffd9000       .debug$S                   0000000180000000     ucrt:api-ms-win-crt-heap-l1-1-0.dll
 0000:fffd9000       .debug$S                   0000000180000000     ucrt:api-ms-win-crt-heap-l1-1-0.dll
 0002:ffffb000       .idata$6                   0000000180000000     ucrt:api-ms-win-crt-heap-l1-1-0.dll
 0000:fffd9000       .debug$S                   0000000180000000     ucrt:api-ms-win-crt-runtime-l1-1-0.dll
 0000:fffd9000       .debug$S                   0000000180000000     ucrt:api-ms-win-crt-runtime-l1-1-0.dll
 0000:fffd9000       .debug$S                   0000000180000000     ucrt:api-ms-win-crt-runtime-l1-1-0.dll
 0000:fffd9000       .debug$S                   0000000180000000     ucrt:api-ms-win-crt-runtime-l1-1-0.dll
 0000:fffd9000       .debug$S                   0000000180000000     ucrt:api-ms-win-crt-runtime-l1-1-0.dll
 0000:fffd9000       .debug$S                   0000000180000000     ucrt:api-ms-win-crt-runtime-l1-1-0.dll
 0000:fffd9000       .debug$S                   0000000180000000     ucrt:api-ms-win-crt-runtime-l1-1-0.dll
 0000:fffd9000       .debug$S                   0000000180000000     ucrt:api-ms-win-crt-runtime-l1-1-0.dll
 0000:fffd9000       .debug$S                   0000000180000000     ucrt:api-ms-win-crt-runtime-l1-1-0.dll
 0000:fffd9000       .debug$S                   0000000180000000     ucrt:api-ms-win-crt-runtime-l1-1-0.dll
 0000:fffd9000       .debug$S                   0000000180000000     ucrt:api-ms-win-crt-runtime-l1-1-0.dll
 0000:fffd9000       .debug$S                   0000000180000000     ucrt:api-ms-win-crt-runtime-l1-1-0.dll
 0000:fffd9000       .debug$S                   0000000180000000     ucrt:api-ms-win-crt-runtime-l1-1-0.dll
 0000:fffd9000       .debug$S                   0000000180000000     ucrt:api-ms-win-crt-runtime-l1-1-0.dll
 0000:fffd9000       .debug$S                   0000000180000000     ucrt:api-ms-win-crt-runtime-l1-1-0.dll
 0000:fffd9000       .debug$S                   0000000180000000     ucrt:api-ms-win-crt-runtime-l1-1-0.dll
 0000:fffd9000       .debug$S                   0000000180000000     ucrt:api-ms-win-crt-stdio-l1-1-0.dll
 0000:fffd9000       .debug$S                   0000000180000000     ucrt:api-ms-win-crt-stdio-l1-1-0.dll
 0000:fffd9000       .debug$S                   0000000180000000     ucrt:api-ms-win-crt-stdio-l1-1-0.dll
 0000:fffd9000       .debug$S                   0000000180000000     ucrt:api-ms-win-crt-stdio-l1-1-0.dll
 0000:fffd9000       .debug$S                   0000000180000000     ucrt:api-ms-win-crt-stdio-l1-1-0.dll
 0000:fffd9000       .debug$S                   0000000180000000     ucrt:api-ms-win-crt-stdio-l1-1-0.dll
 0000:fffd9000       .debug$S                   0000000180000000     ucrt:api-ms-win-crt-stdio-l1-1-0.dll
 0000:fffd9000       .debug$S                   0000000180000000     ucrt:api-ms-win-crt-stdio-l1-1-0.dll
 0000:fffd9000       .debug$S                   0000000180000000     ucrt:api-ms-win-crt-stdio-l1-1-0.dll
 0000:fffd9000       .debug$S                   0000000180000000     ucrt:api-ms-win-crt-stdio-l1-1-0.dll
 0000:fffd9000       .debug$S                   0000000180000000     ucrt:api-ms-win-crt-string-l1-1-0.dll
 0000:fffd9000       .debug$S                   0000000180000000     ucrt:api-ms-win-crt-string-l1-1-0.dll
 0000:fffd9000       .debug$S                   0000000180000000     ucrt:api-ms-win-crt-string-l1-1-0.dll
 0000:fffd9000       .debug$S                   0000000180000000     ucrt:api-ms-win-crt-string-l1-1-0.dll
 0000:fffd9000       .debug$S                   0000000180000000     ucrt:api-ms-win-crt-string-l1-1-0.dll
 0000:fffd9000       .debug$S                   0000000180000000     ucrt:api-ms-win-crt-string-l1-1-0.dll
 0000:fffd9000       .debug$S                   0000000180000000     ucrt:api-ms-win-crt-string-l1-1-0.dll
 0000:fffd9000       .debug$S                   0000000180000000     ucrt:api-ms-win-crt-string-l1-1-0.dll
 0000:fffd9000       .debug$S                   0000000180000000     kernel32:KERNEL32.dll
 0000:fffd9000       .debug$S                   0000000180000000     kernel32:KERNEL32.dll
 0000:fffd9000       .debug$S                   0000000180000000     kernel32:KERNEL32.dll
 0000:fffd9000       .debug$S                   0000000180000000     kernel32:KERNEL32.dll
 0000:fffd9000       .debug$S                   0000000180000000     kernel32:KERNEL32.dll
 0000:fffd9000       .debug$S                   0000000180000000     kernel32:KERNEL32.dll
 0000:fffd9000       .debug$S                   0000000180000000     kernel32:KERNEL32.dll
 0000:fffd9000       .debug$S                   0000000180000000     kernel32:KERNEL32.dll
 0000:fffd9000       .debug$S                   0000000180000000     kernel32:KERNEL32.dll
 0000:fffd9000       .debug$S                   0000000180000000     kernel32:KERNEL32.dll
 0000:fffd9000       .debug$S                   0000000180000000     kernel32:KERNEL32.dll
 0000:fffd9000       .debug$S                   0000000180000000     kernel32:KERNEL32.dll
 0000:fffd9000       .debug$S                   0000000180000000     kernel32:KERNEL32.dll
 0000:fffd9000       .debug$S                   0000000180000000     kernel32:KERNEL32.dll
 0000:fffd9000       .debug$S                   0000000180000000     kernel32:KERNEL32.dll
 0000:fffd9000       .debug$S                   0000000180000000     kernel32:KERNEL32.dll
 0000:fffd9000       .debug$S                   0000000180000000     kernel32:KERNEL32.dll
 0000:fffd9000       .debug$S                   0000000180000000     kernel32:KERNEL32.dll
 0000:fffd9000       .debug$S                   0000000180000000     kernel32:KERNEL32.dll
 0000:fffd9000       .debug$S                   0000000180000000     kernel32:KERNEL32.dll
 0000:fffd9000       .debug$S                   0000000180000000     kernel32:KERNEL32.dll
 0000:fffd9000       .debug$S                   0000000180000000     kernel32:KERNEL32.dll
 0000:fffd9000       .debug$S                   0000000180000000     kernel32:KERNEL32.dll
 0000:fffd9000       .debug$S                   0000000180000000     kernel32:KERNEL32.dll
 0000:fffd9000       .debug$S                   0000000180000000     kernel32:KERNEL32.dll
 0000:fffd9000       .debug$S                   0000000180000000     kernel32:KERNEL32.dll
 0000:fffd9000       .debug$S                   0000000180000000     kernel32:KERNEL32.dll
 0000:fffd9000       .debug$S                   0000000180000000     kernel32:KERNEL32.dll
 0001:00000310       ?check_jvmti_status@@YAXPEAUJNIEnv_@@W4jvmtiError@@PEBD@Z 0000000180001310 f   libpopframe004.obj
 0001:0000055c       ?print_method@@YAXPEAU_jvmtiEnv@@PEAUJNIEnv_@@PEAU_jmethodID@@H@Z 000000018000155c f   libpopframe004.obj
 0001:00000754       ?print_stack_trace@@YAXPEAU_jvmtiEnv@@PEAUJNIEnv_@@PEAV_jobject@@@Z 0000000180001754 f   libpopframe004.obj
 0001:000016a4       addRefToVerify             00000001800026a4 f   libpopframe004.obj
 0001:00001710       agentThreadWrapper         0000000180002710 f   libpopframe004.obj
 0001:00001900       file_basename              0000000180002900 f   libpopframe004.obj
 0001:000020b8       startAgentThreadWrapper    00000001800030b8 f   libpopframe004.obj
 0001:000024a0       syncDebuggeeStatus         00000001800034a0 f   libpopframe004.obj
 0001:00002740       capture_previous_context   0000000180003740 f   MSVCRT:gs_report.obj
 0001:000027b4       ?__scrt_initialize_thread_safe_statics@@YAHXZ 00000001800037b4 f   MSVCRT:thread_safe_statics.obj
 0001:00002884       ?__scrt_uninitialize_thread_safe_statics@@YAXXZ 0000000180003884 f   MSVCRT:thread_safe_statics.obj
 0001:00002aa0       $$000000                   0000000180003aa0     MSVCRT:amdsecgs.obj
 0001:00002ad0       ?dllmain_crt_dispatch@@YAHQEAUHINSTANCE__@@KQEAX@Z 0000000180003ad0 f   MSVCRT:dll_dllmain.obj
 0001:00002b20       ?dllmain_crt_process_attach@@YAHQEAUHINSTANCE__@@QEAX@Z 0000000180003b20 f   MSVCRT:dll_dllmain.obj
 0001:00002c38       ?dllmain_crt_process_detach@@YAH_N@Z 0000000180003c38 f   MSVCRT:dll_dllmain.obj
 0001:00002cbc       ?dllmain_dispatch@@YAHQEAUHINSTANCE__@@KQEAX@Z 0000000180003cbc f   MSVCRT:dll_dllmain.obj
 0001:000036d0       $$000000                   00000001800046d0     MSVCRT:guard_dispatch.obj
 0001:000036f0       $$000000                   00000001800046f0     MSVCRT:guard_xfg_dispatch.obj
 0001:00003706       ?fin$0@?0??dllmain_crt_process_attach@@YAHQEAUHINSTANCE__@@QEAX@Z@4HA 0000000180004706 f   MSVCRT:dll_dllmain.obj
 0001:0000371d       ?fin$0@?0??dllmain_crt_process_detach@@YAH_N@Z@4HA 000000018000471d f   MSVCRT:dll_dllmain.obj
 0001:00003736       ?fin$1@?0??dllmain_crt_process_detach@@YAH_N@Z@4HA 0000000180004736 f   MSVCRT:dll_dllmain.obj
 0001:0000374a       ?filt$0@?0??dllmain_dispatch@@YAHQEAUHINSTANCE__@@KQEAX@Z@4HA 000000018000474a f   MSVCRT:dll_dllmain.obj
 0001:00003780       __scrt_is_nonwritable_in_current_image$filt$0 0000000180004780 f   MSVCRT:utility.obj
 0002:00000208       ?__scrt_initialize_tss_var@@3P6AHXZEA 0000000180005208     MSVCRT:thread_safe_statics.obj
 0002:00000330       ?opcLengths@@3QBEB         0000000180005330     libpopframe004.obj
 0002:00002180       GS_ExceptionPointers       0000000180007180     MSVCRT:gs_report.obj
 0002:00002818       $unwind$fprintf            0000000180007818     libpopframe004.obj
 0002:00002824       $unwind$printf             0000000180007824     libpopframe004.obj
 0002:00002830       $unwind$?CallVoidMethod@JNIEnv_@@QEAAXPEAV_jobject@@PEAU_jmethodID@@ZZ 0000000180007830     libpopframe004.obj
 0002:00002830       $unwind$?NewObject@JNIEnv_@@QEAAPEAV_jobject@@PEAV_jclass@@PEAU_jmethodID@@ZZ 0000000180007830     libpopframe004.obj
 0002:00002830       $unwind$nsk_lcomplain      0000000180007830     libpopframe004.obj
 0002:00002830       $unwind$nsk_ldisplay       0000000180007830     libpopframe004.obj
 0002:00002838       $unwind$nsk_lvdisplay      0000000180007838     libpopframe004.obj
 0002:00002838       $unwind$_RTC_Initialize    0000000180007838     MSVCRT:initsect.obj
 0002:00002838       $unwind$_RTC_Terminate     0000000180007838     MSVCRT:initsect.obj
 0002:00002838       $unwind$?__scrt_initialize_thread_safe_statics@@YAHXZ 0000000180007838     MSVCRT:thread_safe_statics.obj
 0002:00002844       $unwind$nsk_lvcomplain     0000000180007844     libpopframe004.obj
 0002:0000285c       $unwind$nsk_ltrace         000000018000785c     libpopframe004.obj
 0002:0000285c       $unwind$__report_gsfailure 000000018000785c     MSVCRT:gs_report.obj
 0002:00002864       $unwind$Agent_Initialize   0000000180007864     libpopframe004.obj
 0002:00002864       $unwind$nsk_lvtrace        0000000180007864     libpopframe004.obj
 0002:00002864       $unwind$resThread          0000000180007864     libpopframe004.obj
 0002:00002864       $unwind$suspThread         0000000180007864     libpopframe004.obj
 0002:00002864       $unwind$__raise_securityfailure 0000000180007864     MSVCRT:gs_report.obj
 0002:00002864       $unwind$_Init_thread_footer 0000000180007864     MSVCRT:thread_safe_statics.obj
 0002:00002864       $unwind$_Init_thread_header 0000000180007864     MSVCRT:thread_safe_statics.obj
 0002:00002864       $unwind$_Init_thread_wait  0000000180007864     MSVCRT:thread_safe_statics.obj
 0002:00002864       $unwind$__scrt_initialize_crt 0000000180007864     MSVCRT:utility.obj
 0002:00002864       $unwind$__scrt_initialize_onexit_tables 0000000180007864     MSVCRT:utility.obj
 0002:00002864       $unwind$__scrt_release_startup_lock 0000000180007864     MSVCRT:utility.obj
 0002:00002864       $unwind$__scrt_uninitialize_crt 0000000180007864     MSVCRT:utility.obj
 0002:00002864       $unwind$_onexit            0000000180007864     MSVCRT:utility.obj
 0002:0000286c       $unwind$nsk_lverify        000000018000786c     libpopframe004.obj
 0002:0000287c       $unwind$nsk_vprintf        000000018000787c     libpopframe004.obj
 0002:0000288c       $unwind$nsk_printf         000000018000788c     libpopframe004.obj
 0002:00002894       $unwind$?check_jvmti_status@@YAXPEAUJNIEnv_@@W4jvmtiError@@PEBD@Z 0000000180007894     libpopframe004.obj
 0002:000028a4       $unwind$?print_method@@YAXPEAU_jvmtiEnv@@PEAUJNIEnv_@@PEAU_jmethodID@@H@Z 00000001800078a4     libpopframe004.obj
 0002:000028bc       $unwind$?print_stack_trace@@YAXPEAU_jvmtiEnv@@PEAUJNIEnv_@@PEAV_jobject@@@Z 00000001800078bc     libpopframe004.obj
 0002:000028dc       $unwind$?nsk_jni_lverify@@YAHHPEAUJNIEnv_@@HQEBDH1ZZ 00000001800078dc     libpopframe004.obj
 0002:000028f0       $unwind$?nsk_jni_check_exception@@YAHPEAUJNIEnv_@@QEBDH@Z 00000001800078f0     libpopframe004.obj
 0002:0000290c       $unwind$FramePop           000000018000790c     libpopframe004.obj
 0002:0000290c       $unwind$Java_nsk_jvmti_unit_FollowReferences_FollowRefObjects_resetTags 000000018000790c     libpopframe004.obj
 0002:0000290c       $unwind$MethodExit         000000018000790c     libpopframe004.obj
 0002:0000290c       $unwind$addRefToVerify     000000018000790c     libpopframe004.obj
 0002:0000290c       $unwind$nsk_jvmti_resetAgentData 000000018000790c     libpopframe004.obj
 0002:0000290c       $unwind$nsk_jvmti_setFailStatus 000000018000790c     libpopframe004.obj
 0002:0000290c       $unwind$__scrt_initialize_default_local_stdio_options 000000018000790c     MSVCRT:default_local_stdio_options.obj
 0002:0000290c       $unwind$?dllmain_crt_dispatch@@YAHQEAUHINSTANCE__@@KQEAX@Z 000000018000790c     MSVCRT:dll_dllmain.obj
 0002:0000290c       $unwind$DllMain            000000018000790c     MSVCRT:dll_dllmain_stub.obj
 0002:0000290c       $unwind$__GSHandlerCheck   000000018000790c     MSVCRT:gshandler.obj
 0002:0000290c       $unwind$?__scrt_uninitialize_thread_safe_statics@@YAXXZ 000000018000790c     MSVCRT:thread_safe_statics.obj
 0002:0000290c       $unwind$_Init_thread_notify 000000018000790c     MSVCRT:thread_safe_statics.obj
 0002:0000290c       $unwind$__scrt_acquire_startup_lock 000000018000790c     MSVCRT:utility.obj
 0002:0000290c       $unwind$__scrt_dllmain_after_initialize_c 000000018000790c     MSVCRT:utility.obj
 0002:0000290c       $unwind$__scrt_dllmain_before_initialize_c 000000018000790c     MSVCRT:utility.obj
 0002:0000290c       $unwind$__scrt_dllmain_crt_thread_attach 000000018000790c     MSVCRT:utility.obj
 0002:0000290c       $unwind$__scrt_dllmain_crt_thread_detach 000000018000790c     MSVCRT:utility.obj
 0002:0000290c       $unwind$__scrt_dllmain_uninitialize_c 000000018000790c     MSVCRT:utility.obj
 0002:0000290c       $unwind$__scrt_dllmain_uninitialize_critical 000000018000790c     MSVCRT:utility.obj
 0002:0000290c       $unwind$atexit             000000018000790c     MSVCRT:utility.obj
 0002:00002914       $unwind$nsk_jvmti_lverify  0000000180007914     libpopframe004.obj
 0002:00002928       $unwind$exitOnError        0000000180007928     libpopframe004.obj
 0002:00002938       $unwind$Java_nsk_share_jvmti_ArgumentHandler_getAgentOptionsString 0000000180007938     libpopframe004.obj
 0002:0000294c       $unwind$Java_nsk_jvmti_unit_FollowReferences_FollowRefObjects_getTag 000000018000794c     libpopframe004.obj
 0002:0000294c       $unwind$Java_nsk_share_jvmti_DebugeeClass_checkStatus 000000018000794c     libpopframe004.obj
 0002:0000294c       $unwind$agentThreadWrapper 000000018000794c     libpopframe004.obj
 0002:0000295c       $unwind$startAgentThreadWrapper 000000018000795c     libpopframe004.obj
 0002:00002978       $unwind$syncDebuggeeStatus 0000000180007978     libpopframe004.obj
 0002:00002978       $unwind$__scrt_dllmain_exception_filter 0000000180007978     MSVCRT:utility.obj
 0002:0000298c       $unwind$Java_nsk_share_jvmti_DebugeeClass_resetAgentData 000000018000798c     libpopframe004.obj
 0002:00002994       $unwind$MA_checkStatus     0000000180007994     libpopframe004.obj
 0002:000029a8       $unwind$Java_nsk_jvmti_unit_FollowReferences_FollowRefObjects_setTag 00000001800079a8     libpopframe004.obj
 0002:000029c0       $unwind$Java_nsk_jvmti_unit_FollowReferences_FollowRefObjects_addRefToVerify 00000001800079c0     libpopframe004.obj
 0002:000029dc       $unwind$Java_nsk_jvmti_PopFrame_popframe004_doPopFrame 00000001800079dc     libpopframe004.obj
 0002:000029f4       $unwind$Java_nsk_jvmti_PopFrame_popframe004_nativeMeth 00000001800079f4     libpopframe004.obj
 0002:000029f4       $unwind$nativeMeth2        00000001800079f4     libpopframe004.obj
 0002:000029f4       $unwind$_DllMainCRTStartup 00000001800079f4     MSVCRT:dll_dllmain.obj
 0002:00002a04       $unwind$capture_previous_context 0000000180007a04     MSVCRT:gs_report.obj
 0002:00002a10       $unwind$__GSHandlerCheckCommon 0000000180007a10     MSVCRT:gshandler.obj
 0002:00002a18       $xdatasym                  0000000180007a18     MSVCRT:amdsecgs.obj
 0002:00002a1c       $unwind$?dllmain_crt_process_attach@@YAHQEAUHINSTANCE__@@QEAX@Z 0000000180007a1c     MSVCRT:dll_dllmain.obj
 0002:00002a58       $unwind$?fin$0@?0??dllmain_crt_process_attach@@YAHQEAUHINSTANCE__@@QEAX@Z@4HA 0000000180007a58     MSVCRT:dll_dllmain.obj
 0002:00002a58       $unwind$?fin$0@?0??dllmain_crt_process_detach@@YAH_N@Z@4HA 0000000180007a58     MSVCRT:dll_dllmain.obj
 0002:00002a58       $unwind$?fin$1@?0??dllmain_crt_process_detach@@YAH_N@Z@4HA 0000000180007a58     MSVCRT:dll_dllmain.obj
 0002:00002a60       $unwind$?dllmain_crt_process_detach@@YAH_N@Z 0000000180007a60     MSVCRT:dll_dllmain.obj
 0002:00002ab4       $unwind$?dllmain_dispatch@@YAHQEAUHINSTANCE__@@KQEAX@Z 0000000180007ab4     MSVCRT:dll_dllmain.obj
 0002:00002adc       $unwind$?filt$0@?0??dllmain_dispatch@@YAHQEAUHINSTANCE__@@KQEAX@Z@4HA 0000000180007adc     MSVCRT:dll_dllmain.obj
 0002:00002ae4       $unwind$__scrt_is_nonwritable_in_current_image 0000000180007ae4     MSVCRT:utility.obj
 0002:00002b04       $unwind$__scrt_is_nonwritable_in_current_image$filt$0 0000000180007b04     MSVCRT:utility.obj
 0002:00002b0c       $unwind$__scrt_fastfail    0000000180007b0c     MSVCRT:utility_desktop.obj
 0002:00002b1c       $unwind$__security_init_cookie 0000000180007b1c     MSVCRT:gs_support.obj
 0002:00002b28       $unwind$__isa_available_init 0000000180007b28     MSVCRT:cpu_disp.obj
 0002:00002b38       $xdatasym                  0000000180007b38     MSVCRT:guard_dispatch.obj
 0002:00002b40       $xdatasym                  0000000180007b40     MSVCRT:guard_xfg_dispatch.obj
 0002:00002b50       .edata                     0000000180007b50     popframe004.exp
 0002:00002b78       rgpv                       0000000180007b78     popframe004.exp
 0002:00002bbc       rgszName                   0000000180007bbc     popframe004.exp
 0002:00002c00       rgwOrd                     0000000180007c00     popframe004.exp
 0002:00002c22       szName                     0000000180007c22     popframe004.exp
 0002:00002c32       $N00001                    0000000180007c32     popframe004.exp
 0002:00002c41       $N00002                    0000000180007c41     popframe004.exp
 0002:00002c4e       $N00003                    0000000180007c4e     popframe004.exp
 0002:00002c7d       $N00004                    0000000180007c7d     popframe004.exp
 0002:00002cab       $N00005                    0000000180007cab     popframe004.exp
 0002:00002cda       $N00006                    0000000180007cda     popframe004.exp
 0002:00002d1f       $N00007                    0000000180007d1f     popframe004.exp
 0002:00002d5c       $N00008                    0000000180007d5c     popframe004.exp
 0002:00002da4       $N00009                    0000000180007da4     popframe004.exp
 0002:00002de4       $N00010                    0000000180007de4     popframe004.exp
 0002:00002e21       $N00011                    0000000180007e21     popframe004.exp
 0002:00002e5c       $N00012                    0000000180007e5c     popframe004.exp
 0002:00002e8a       $N00013                    0000000180007e8a     popframe004.exp
 0002:00002ebb       $N00014                    0000000180007ebb     popframe004.exp
 0002:00002eea       $N00015                    0000000180007eea     popframe004.exp
 0002:00002f19       $N00016                    0000000180007f19     popframe004.exp
 0002:00002f4e       $N00017                    0000000180007f4e     popframe004.exp
 0002:000033dc       .idata$6                   00000001800083dc     kernel32:KERNEL32.dll
 0002:00003440       .idata$6                   0000000180008440     vcruntime:VCRUNTIME140.dll
 0002:000035a2       .idata$6                   00000001800085a2     ucrt:api-ms-win-crt-runtime-l1-1-0.dll
 0002:000035c4       .idata$6                   00000001800085c4     ucrt:api-ms-win-crt-stdio-l1-1-0.dll
 0002:000035e4       .idata$6                   00000001800085e4     ucrt:api-ms-win-crt-string-l1-1-0.dll
 0003:00000000       ?UNNAMED_STR@?1??get_thread_name@@YAPEADPEAU_jvmtiEnv@@PEAUJNIEnv_@@PEAV_jobject@@@Z@4PEBDEB 0000000180009000     libpopframe004.obj
 0003:00000008       ?codeAttributeName@@3PEBDEB 0000000180009008     libpopframe004.obj
 0003:00000010       ?lineNumberAttributeName@@3PEBDEB 0000000180009010     libpopframe004.obj
 0003:00000018       ?localVarAttributeName@@3PEBDEB 0000000180009018     libpopframe004.obj
 0003:00000020       ?localVarTypeAttributeName@@3PEBDEB 0000000180009020     libpopframe004.obj
 0003:00000028       ?stackMapAttributeName@@3PEBDEB 0000000180009028     libpopframe004.obj
 0003:00000030       ?callBytes@@3PAEA          0000000180009030     libpopframe004.obj
 0003:00000034       ?allocBytes@@3PAEA         0000000180009034     libpopframe004.obj
 0003:0001aad4       redefineAttempted          0000000180023ad4     libpopframe004.obj
 0003:0001aad8       nsk_context                0000000180023ad8     libpopframe004.obj
 0003:0001aae4       redefineSucceed            0000000180023ae4     libpopframe004.obj
 0003:0001aae8       agentFailed                0000000180023ae8     libpopframe004.obj
 0003:0001aaec       currentAgentStatus         0000000180023aec     libpopframe004.obj
 0003:0001aaf0       context                    0000000180023af0     libpopframe004.obj
 0003:0001aba8       agentThread                0000000180023ba8     libpopframe004.obj
 0003:0001abb0       agentThreadProc            0000000180023bb0     libpopframe004.obj
 0003:0001abb8       agentThreadArg             0000000180023bb8     libpopframe004.obj
 0003:0001abc0       agent_data                 0000000180023bc0     libpopframe004.obj
 0003:0001abd0       jvmti_env                  0000000180023bd0     libpopframe004.obj
 0003:0001abd8       jvm                        0000000180023bd8     libpopframe004.obj
 0003:0001abe0       jni_env                    0000000180023be0     libpopframe004.obj
 0003:0001abe8       checkStatus_func           0000000180023be8     libpopframe004.obj
 0003:0001abf0       ?codeAttributeIndex@@3GA   0000000180023bf0     libpopframe004.obj
 0003:0001abf4       ?lineNumberAttributeIndex@@3GA 0000000180023bf4     libpopframe004.obj
 0003:0001abf8       ?localVarAttributeIndex@@3GA 0000000180023bf8     libpopframe004.obj
 0003:0001abfc       ?localVarTypeAttributeIndex@@3GA 0000000180023bfc     libpopframe004.obj
 0003:0001ac00       ?stackMapAttributeIndex@@3GA 0000000180023c00     libpopframe004.obj
 0003:0001ac04       ?stackFrameOffset@@3GA     0000000180023c04     libpopframe004.obj
 0003:0001ac08       ?mode@@3HA                 0000000180023c08     libpopframe004.obj
 0003:0001ac0c       ?constantPoolSize@@3GA     0000000180023c0c     libpopframe004.obj
 0003:0001ac10       ?orig@@3PEBEEB             0000000180023c10     libpopframe004.obj
 0003:0001ac18       ?gen@@3PEAEEA              0000000180023c18     libpopframe004.obj
 0003:0001ac20       ?inputPos@@3PEAEEA         0000000180023c20     libpopframe004.obj
 0003:0001ac28       ?endPos@@3PEBEEB           0000000180023c28     libpopframe004.obj
 0003:0001ac30       ?genPos@@3PEAEEA           0000000180023c30     libpopframe004.obj
 0003:0001ac38       ?markPos@@3PEAEEA          0000000180023c38     libpopframe004.obj
 0003:0001ac40       ?constantPool@@3PEAPEADEA  0000000180023c40     libpopframe004.obj
 0003:0001ac48       ?constantPoolCount@@3GA    0000000180023c48     libpopframe004.obj
 0003:0001ac4c       ?zeroBytes@@3PAEA          0000000180023c4c     libpopframe004.obj
 0003:0001ac50       ?codeLength@@3IA           0000000180023c50     libpopframe004.obj
 0003:0001ac54       watch_ev                   0000000180023c54     libpopframe004.obj
 0003:0001ac58       ?map@@3PEAIEA              0000000180023c58     libpopframe004.obj
 0003:0001ac60       ?widening@@3PEACEA         0000000180023c60     libpopframe004.obj
 0003:0001ac68       jvmti                      0000000180023c68     libpopframe004.obj
 0003:0001ac70       caps                       0000000180023c70     libpopframe004.obj
 0003:0001ac80       callbacks                  0000000180023c80     libpopframe004.obj
 0003:0001adb8       gen_ev                     0000000180023db8     libpopframe004.obj
 0003:0001adbc       popDone                    0000000180023dbc     libpopframe004.obj
 0003:0001adc0       tot_result                 0000000180023dc0     libpopframe004.obj
 0003:0001adc8       watch_ev_monitor           0000000180023dc8     libpopframe004.obj
 0003:0001add8       ?UNNAMED_LEN@?1??get_thread_name@@YAPEADPEAU_jvmtiEnv@@PEAUJNIEnv_@@PEAV_jobject@@@Z@4_KA 0000000180023dd8     libpopframe004.obj
 0003:0001ade0       ?$TSS0@?1??get_thread_name@@YAPEADPEAU_jvmtiEnv@@PEAUJNIEnv_@@PEAV_jobject@@@Z@4HA 0000000180023de0     libpopframe004.obj
 0003:0001adf0       GS_ExceptionRecord         0000000180023df0     MSVCRT:gs_report.obj
 0003:0001ae90       GS_ContextRecord           0000000180023e90     MSVCRT:gs_report.obj
 0003:0001b360       ?g_tss_cv@@3U_RTL_CONDITION_VARIABLE@@A 0000000180024360     MSVCRT:thread_safe_statics.obj
 0003:0001b368       ?g_tss_event@@3PEAXEA      0000000180024368     MSVCRT:thread_safe_statics.obj
 0003:0001b370       ?g_tss_mutex@@3U_RTL_CRITICAL_SECTION@@A 0000000180024370     MSVCRT:thread_safe_statics.obj
 0003:0001b398       ?g_sleep_condition_variable_cs@@3P6AHPEAU_RTL_CONDITION_VARIABLE@@PEAU_RTL_CRITICAL_SECTION@@K@ZEA 0000000180024398     MSVCRT:thread_safe_statics.obj
 0003:0001b3a0       ?g_wake_all_condition_variable@@3P6AXPEAU_RTL_CONDITION_VARIABLE@@@ZEA 00000001800243a0     MSVCRT:thread_safe_statics.obj
 0003:0001b3ac       ?__proc_attached@@3HA      00000001800243ac     MSVCRT:dll_dllmain.obj
 0003:0001b3c0       ?is_initialized_as_dll@@3_NA 00000001800243c0     MSVCRT:utility.obj
 0003:0001b3c1       ?module_local_atexit_table_initialized@@3_NA 00000001800243c1     MSVCRT:utility.obj
 0003:0001b3c8       ?module_local_atexit_table@@3U_onexit_table_t@@A 00000001800243c8     MSVCRT:utility.obj
 0003:0001b3e0       ?module_local_at_quick_exit_table@@3U_onexit_table_t@@A 00000001800243e0     MSVCRT:utility.obj
